:020000040000FA
:10000000BB2A29205320282088010B114508463E91
:10001000840022008D122A308C0518308D052000B6
:10002000C20B19321030C200073021008D042000AD
:100030000D080D080D080D080D080D080D080739ED
:10004000C1002100F8308D052000CD08031DCD032F
:10005000C408031DC40322004620C639801F013E88
:100060008D04462019398919091589118C047B20C2
:100070008C0420398D042000C50A4508023C031C6D
:10008000C501C3030319AE15CE0A090000087F3964
:100090002C3C00087F39031C2A3082073034F634A8
:1000A000A834A434663425342134B63420342434BE
:1000B000223461343934E03429342B346234FB3453
:1000C000F0346B3479343234E334E1342A34EB34B1
:1000D00027346934F13470346434E634FF34BF3487
:1000E000EF34FD34ED34AD342E34E934B4347234AD
:1000F000FD34FD34FD3420004508220003390B0097
:100100002034403480342034A53007328A30053220
:10011000123003320B30013201306400A701A60017
:10012000A60BFE332708031908006400A703F83361
:100130001508C039031DFC3308000530A0002E113E
:10014000982022008D1121008D1120008420210093
:100150008D15200088208D192E1586202E1D080053
:10016000A00BEE3308000830AA00982022008D1161
:1001700021008D110032003200008D1520008C20EE
:10018000003203108D190314AF0C8A20AA0BF03330
:100190002F080800AF010230E733AF000830AA0093
:1001A000982022008D112000AF0C21008D1120001D
:1001B000031C8820003221008D15200003188820A0
:1001C0008C20AA0BF13308000130E9332F08A90075
:1001D0000830AA00A90C03180732B01B073203101D
:1001E000B00DAA0BF7330800B01BF9331830B00676
:1001F0000314B00DF6332830A1000830A000CA2047
:100200002108AF00E420A10CA00BF9330800B101D4
:10021000A9019D20F030CD20FB202908FC20CA2018
:1002200003191732C03A03190D323108333E8600E4
:1002300029088100B10A3108803EC600023031022F
:1002400003180800A90FE533B308031D0800C8010F
:1002500002320230C800C7018E30C60008006400B8
:1002600021009D182B321B082000BD0721001C080F
:100270002000BE3D0301BF3D21009D142000C00BA6
:100280001D323E08A0003F08A100BD01BE01BF0114
:10029000A201C830A300A401A5012F222608A000B6
:1002A0002708A1002808A200A930A3000230A4005A
:1002B000FA212608BB002708BC0008002000CD0852
:1002C000031D0800D9212E195232BE30CD20B001B5
:1002D000B320A300E620B320A400E6200730A0004E
:1002E000B320E620A00BFC33B00803190232F4213E
:1002F0003E325022A0002408A10050225022A00724
:100300000318A10A2408A107200EF038A000210E2E
:100310000F38A005210E0F39A11BF038A100033AB8
:10032000031D18322008523A031D14320310310DF8
:10033000373E86000108A000860A0108A1003E3071
:10034000A3000330A400B623031C11325230A000D6
:100350000330A1000310310D373E860020088100D4
:10036000860A210881003108353E86008101B10AE4
:1003700032083102031C0132B101D9212E19163283
:10038000B430CD208D1121008D1100008D1520007D
:10039000AE128D19AE16D9212E1908324430CD2057
:1003A000AE1A04328D1521008D1120001830CD00B9
:1003B000C72B9D202E191832F030CD20FB2031089C
:1003C000333E86000108FC203030A000CA2003190B
:1003D0000B32C03A0319083203012F1B0130AF0062
:1003E000E420A00BF33308003108353E8600011DE0
:1003F000810A08002008A9002108AA002208AB00F1
:10040000A001A101A2011830AC0003101822031CA6
:100410000532A2002708A1002608A000AC0BF63385
:10042000290DA6002A0DA7002B0DA8000311080016
:10043000A90DAA0DAB0DA00DA10DA20D2308200240
:10044000A6002408213BA7002508223BA80008009D
:100450002008A6072108A73D2208A83D080020087B
:10046000A9002108AA002208AB00A601A701A80143
:1004700003101930AC00A50CA40CA30C0308AD00AC
:1004800003182822A00DA10DA20D2D088300AC0B8E
:10049000F2332908A0002A08A1002B08A2000800B6
:1004A0000310A30DA40D23080800A000343E86000D
:1004B00001194732200386000310060D373E8600DF
:1004C0000108A000860A0108A100AE13A11F063290
:1004D000AE17A109A009A00F0132A10AA201E830BC
:1004E000A3000330A400A501FA212608CC00643043
:1004F000A300A401FA212608CB000A30A300A4011E
:10050000FA212608CA002008C900AE1B1532CC0803
:10051000031D0A324B0803192030C6004A08803EEA
:10052000C7004908C80008004C08C6004B08C700AF
:100530004A08803EC80008002230CB08031DF5336E
:10054000EC330E30C6009930C7002003C800080005
:1005500064004108073A031D03322E12AE1508004D
:100560000315AE1D080018302E1EF430C300AE1166
:100570002E16031108002300E2308C0001308D009C
:100580002200403097005A309800F730990021003F
:100590006F30990022308C0008308D004330950078
:1005A00087309D00A8309E00200020308B009801ED
:1005B0009C01850187010730C100C201C5010D12F0
:1005C0008C11BD01BE01BF01C0018B1764008030DA
:1005D000C6000D30C7001A30C80007210F30C40014
:1005E0006400C408031DFC3346088E3A0319EE3339
:1005F0003108B200BC210D168C1100303C23AE1521
:10060000D630C400A822031D5C322F21AE184E1F25
:1006100006322030C600C800803EC70002320130DA
:100620005522C408031DEE330D128C1501303C23F6
:10063000AE15D630C400A822031D64322F2102302B
:100640005522C408031DF7330D168C151D303C23AD
:10065000AE15D630C400A822031D6C322F213B08F2
:10066000A0003C08A1006522C408031DF433320831
:10067000023C0319C033AA33C8002030C600C700AB
:100680000A30C400A822031D0800C408031DFA3361
:100690004808C7002030C8000A30C400A822031D43
:1006A0000800C408031DFA334708C6002030C700FD
:1006B0000A30C400A822031D0800C408031DFA3331
:1006C00008000030C6001C30C7001B30C8000D16E3
:1006D0008C11C3016400AE1D0232AE118C3341088F
:1006E000073A031DF7332F21AE184E1F0632203074
:1006F000C600C800803EC700023201305522A82241
:100700000319F1330130C6001630C7002030C8008D
:100710000D128C15C3016400AE1D0232AE116B3395
:100720004108073A031DF7332F2102305522A82232
:100730000319FA330B30C6000A30C7001B30C8005B
:100740000D168C15C3016400AE1D0232AE11533379
:100750004108073A031DF7332F213B08A0003C084E
:10076000A1006522A8220319F733AB332108240620
:100770008039240D031D0800A201A5011E22A8082E
:100780000319A7080319A608031903100800AE10DF
:10079000351908003708A0003808A1000A30A30066
:1007A000A401B623031808003708A3003808A400E2
:1007B000F630A000FF30A100B623031CAE140800E1
:020000040001F9
:02000E009C0F45
:02001000FF3CB3
:00000001FF
